:020000020000FC
:1000000002C60CC0000000000EC10000E6C00000E7
:10001000E8C09AC000000000000000001FB64CB508
:100020005DB591FD23C097FF62E097FD63E065BF7A
:100030009260C0B297FDC094C2FE03C0742E852E9C
:100040007EC097FF63E097FD62E065BF662760644E
:100050006ABF9D7F40E050E0C0B297FDC094C2FCF3
:1000600067C050937C0040937B0062C097FF63E0C1
:1000700097FD62E065BF9D7F83FF3BC097FF62E015
:1000800097FD63E065BF662760646ABF9260409336
:10009000790050937A0060917700B0907800461B09
:1000A0005B09B02C443B60E0560720F46627606291
:1000B000B62E17C0483661E0560720F46627606107
:1000C000B62E0FC0403D62E0560720F466276860F8
:1000D000B62E07C0403A65E0560718F466276460FC
:1000E000B62E4091790050917A004093770050935A
:1000F00078004719580995FD09C094FD09C0569527
:10010000479593FD05C05695479502C0440F551F6E
:100110004A3F500508F04AEF50917B0050937C0015
:1001200040937B0083FF04C06CE3609596239B297A
:1001300040E2D42E916083FD02C050E05BBF50E1ED
:10014000E52E1FBE189518951FB6DD2011F0DA9424
:100150001EC040E050E060B397FD609562FD4AEF3D
:1001600097FF63E097FD62E065BF662760646ABF42
:100170009D7F60B397FD609562FD5AEF451749F783
:1001800050E2D52E40937C0040937B009160EE209E
:1001900011F0EA9405C050E45BBF552750645ABF84
:1001A00090FF19C050917C0040917B0095FD450F58
:1001B00095FD47959E7F50918A00451710F4409118
:1001C0008A00572F507F552331F4242E4091880008
:1001D000433008F0422C1FBE18951FB67E7F1FBE0D
:1001E00018951FB652E040917B00415018F00092E4
:1001F0007E0009C040917E004F3F29F040917E0073
:10020000439540937E0060918800623011F4209005
:100210006D00321431F010F03A9401C033945A95C5
:1002200091F71FBE18951FB6601421F064BC6624B8
:100230001FBE189581FF0994452D089496FF440F21
:1002400010F0642E40E044BD58B18D7F652D6A3FAB
:1002500070F448B3487F48BB82FF09C042E04A952A
:10026000F1F742B3486342BB816055FF8E7F1FBEEA
:100270001895826042C0C098C29A82603EC0C19800
:10028000C09A82603AC0C298C19A826036C04FE07C
:10029000959894984A95E1F7C098C29A82602DC0CB
:1002A0004FE0959893984A95E1F7C098C29A82607A
:1002B00024C04FE0939895984A95E1F7C198C09A69
:1002C00082601BC04FE0939894984A95E1F7C198DB
:1002D000C09A826012C04FE0949893984A95E1F7D3
:1002E000C298C19A826009C04FE0949895984A9547
:1002F000E1F7C298C19A826000C0452D40950894EC
:1003000096FF440F10F0642E40E044BD1FBE1895C8
:100310000000089521E00AC023E008C02AE006C0DA
:100320002EE104C024E602C028EC00C014E000EC7A
:10033000EFDF0A95E9F71A95D1F72A95B9F70895ED
:1003400035E120E509C032E124E606C03FE028E7B8
:1003500003C03CE02CE800C0939A06E90A95F1F747
:100360000CE0C29AD5DF0A95E9F7C29810E4032F92
:10037000CFDF0A95E9F71A95D1F72A9569F793988F
:10038000089500918800033008F028C000916300B0
:100390001091640022E00038120770F0422C0092A5
:1003A000650000926600009267000092680000926B
:1003B000690000926E0012C0232D2095221F221F7B
:1003C000322F2795317033952E7F2054300920939A
:1003D00065003093660001E000936E00089500917F
:1003E0006E000015E1F0009165001091660020910B
:1003F000630030916400021B130B2FEF00381207CB
:1004000044F020E00F3712070CF405C00FE710E0AE
:1004100002C000E81FEF00936A0010936B0008957C
:1004200000916E00001581F1209167003091680005
:100430009090690000916A0010916B00200F311FAD
:10044000911E10EF91164CF01FE091160CF409C0AC
:100450002FEF3FEF1FE0912E04C020E030E010EFBF
:10046000912E10917F004116142D18F4113020F0B8
:1004700005C000234AF002C0002332F42093670035
:100480003093680090926900089500916E00001505
:10049000E9F100916A00112707FD1095000F111F67
:1004A0003091860030FD05C0343089F015950795F0
:1004B0000EC0A12E902EA5949794090D1A1D3530CB
:1004C00031F015950795333011F0159507952FEFFD
:1004D0000038120744F020E00F3712070CF405C073
:1004E0000FE710E002C000E81FEF232D00233AF0D1
:1004F000201B18F0213008F007C021E005C001954D
:10050000200F08F001C02FEF20936C000895009198
:100510006E000015D9F110916800209169003091AA
:10052000870030FD05C0343089F0259517950EC041
:10053000A22E912EA5949794190D2A1D353031F0D5
:1005400025951795333011F0259517950FEF10303D
:10055000200744F000E01F3F20070CF405C01FEF08
:1005600020E002C010E02FEF00916C0022233AF04F
:10057000011B18F0013008F008C001E006C010951A
:100580001395010F08F001C00FEF402E089500EC05
:1005900007B906B10068006406B926B126FDF7CF99
:1005A00004B115B126B12F7726B923ED2093810030
:1005B00020E02093820021E02093800023ED30E0B2
:1005C000220F331F02171307C8F0209381003093C6
:1005D000820022E02093800023ED30E0922EA32EB3
:1005E000220F331F290D3A1D0217130738F02093ED
:1005F00081003093820023E020938000089500EC76
:1006000007B906B10068006406B9089526B126FD51
:10061000FDCF04B115B126B12F7726B90F3F23E0E6
:10062000120778F42091810030918200021713079D
:1006300040F400917F00002359F00A9500937F0059
:1006400007C000917F000F3F19F0039500937F00D2
:10065000401608F4042D502E089574FD02E375FD34
:1006600000E576FD00E577FD08E2172F107F1123E6
:1006700099F020918B00233061F0102F169520FD0A
:1006800001C0169522FD02C0011B03C0010F08F432
:100690000FEF202E402E502E0895C8EBDBE0C093C4
:1006A0007500D09376002FEF3FE1209373003093D5
:1006B000740020936F003093700036952795209337
:1006C0007100309372001FEF109364000FEF0093DE
:1006D00063000895C0917500D091760004C0C09168
:1006E0006F00D0917000F8940CB51DB5C00FD11FEC
:1006F000DBBDCABD789471602091610030916200C9
:100700000093610010936200021B130B20916300A1
:1007100030916400E901D695C795D695C7952C1BF5
:100720003D0B200F311F209363003093640008F0CD
:1007300008951FEF109364000FEF00936300089576
:1007400070FDFECFC0917100D0917200F8940CB58D
:100750001DB50C0F1D1F1BBD0ABD78947160089557
:100760000091630010916400169507951695079502
:1007700016950795169507950550100918F0053040
:10078000100510F405E01127009373001093740016
:1007900000936F00109370001695079500937100F9
:1007A00010937200089570FDFECFC0916300D09148
:1007B0006400F8940CB51DB50C0F1D1F1BBD0ABDC0
:1007C000789471600895789470FF089582FD01C057
:1007D00004C080FDF8CF7894089506E0252D20957B
:1007E0002295269527702395F8940A95F1F718B16C
:1007F00015FDE9CF2A95D9F778940895789470FF7C
:10080000089582FD01C004C080FFF8CF7894089558
:1008100006E0252D20952295269527702395F8949E
:100820000A95F1F718B115FFE9CF2A95D9F7789411
:100830000895C0917300D0917400F8940CB51DB563
:100840000C0F1D1F1BBD0ABD78947160089570FDCB
:10085000FECF0895F894ABE6B1E0FD019398959A28
:1008600002E007B978940895F894A2E6B1E0FD019A
:10087000C19881FDC09A04E007B978940895F8946E
:10088000A9E5B1E0FD019598949A05E007B978943F
:100890000895F894A0E5B1E0FD01C09881FDC29AE9
:1008A00002E007B978940895F894A7E4B1E0FD0157
:1008B0009498939A04E007B978940895F894A4E77B
:1008C000B1E0FD01C29881FDC19A05E007B97894B5
:1008D0000895F8949398959A02E007B9789408954A
:1008E000F894AFE3B1E0FD01C19881FDC09A04E046
:1008F00007B978940895F8949598949A05E007B903
:1009000078940895F894ABE3B1E0FD01C09881FDBF
:10091000C29A02E007B978940895F8949498939A4B
:1009200004E007B978940895F894A3E4B1E0FD01D8
:10093000C29881FDC19A05E007B978940895A9E3AA
:10094000B1E0FD0108B3087F08BB02B3077C02BB1E
:1009500008950091750010917600083E23E012077B
:1009600008F408950091750010917600055010402C
:100970000093750010937600089570FDFECF0895E2
:1009800004E00093860004E00093870001E00093F8
:10099000880003E000938B0090649F770895E199AD
:1009A000FECF1EBB2FBBE09A0DB30895E199FECF99
:1009B0000DBB1EBB2FBBF894E29AE19A7894089580
:1009C00018E020E00FEFF2DF19E020E00FEFEEDF9C
:1009D000089518E020E005EAE9DF19E020E00AE5E3
:1009E000E5DF089518E020E0DADF053A31F519E097
:1009F00020E0D5DF0A3509F510E020E0D0DF0093D4
:100A0000860011E020E0CBDF0093870012E020E0B9
:100A1000C6DF0093880015E020E0C1DF00938B0063
:100A200016E020E0BCDF906401FD9F7B17E020E032
:100A3000B6DF9F7701FD906802C0A2DF01D0089564
:100A4000BFDF01E0009383000091860000938400E3
:100A50002CD002E000938300009187000093840073
:100A600024D003E000938300009188000093840069
:100A70001CD004E00093830000918B00009384005D
:100A800014D005E00093830001E096FF02E000939C
:100A900084000BD006E00093830001E097FD02E0A4
:100AA0000093840002D095DF089530918300009177
:100AB0008400313051F0323061F0333071F0343035
:100AC00081F0353091F03630A1F010E020E06EDF9B
:100AD00014C011E020E06ADF10C012E020E066DF01
:100AE0000CC015E020E062DF08C016E020E05EDF09
:100AF00004C017E020E05ADF00C0089505E0902E02
:100B000013DC9A94E9F70895F8941ADC1CDC1EDCD7
:100B100020DC04DC15DC17DC19DC1BDCFFDB10DC63
:100B200012DC14DC16DC7894089590908300A09079
:100B30008400F89405DC04DC03DCF0DB9A94D1F744
:100B400008DCECDBAA94E1F778940895F89401DCD2
:100B50007894E8DB00917B000130C0F7F894F0DB7B
:100B6000DDDBEEDB7894DEDB00917B000A3FB0F347
:100B7000CBDFC4DFC3DF01E00093830001E000931B
:100B8000840000E000938500D0DF05E0902ECCDBF0
:100B900000917B00013040F413DF87DF1ADFB4DF00
:100BA00008E000932100AADF9A9489F7009185005C
:100BB000039500938500033008F4E6CF9FDF009192
:100BC000840003950093840015E0009183000330B6
:100BD00009F413E000918300053008F012E013954A
:100BE00000918400011708F4CCCF88DF87DF0091E3
:100BF0008300039500938300073008F4BFCF08E01B
:100C0000009321007BDFF894A89501B5086101BD30
:100C100000E001BD04E00EBF0FE50DBF90DE00E077
:100C200008BB07E107BB00E005BB00E004BB00E038
:100C300002BB08E301BB0024A0E0B0E00D92AA31A2
:100C4000E9F7A0E6B0E004E60D920A95E9F777DE51
:100C500002E003BF02E00EBD01E005BD91DEC2DE91
:100C600063DB6EDB5DDB6FDB5BDB70DB59DB05E5DC
:100C700008BF09BF06B10260016006B9789487DC3D
:100C800097FF03E097FD02E005BF00E40BBF0027DC
:100C900000640ABF9D7F48DB3FDB00917B00013091
:100CA000D8F742DB886015E0912E36DB90FFFECF4F
:100CB00000917B000230B8F3292F2C7330917D0016
:100CC00020937D00231779F79A9479F7877F97FF10
:100CD00003E097FD02E005BF002700640ABF9D7F87
:100CE000F8942EDB2DDB2CDB78941EDB00926D005C
:100CF00013DB00917B000A3F08F028CF10916D00B4
:100D0000011710F000936D00013090F7F89421DB8B
:100D100020DB1FDB789408DBFFDA00917B000130D9
:100D2000D8F30DDE22243324442455240FEF0093FE
:100D30007F000092650000926600009267000092BA
:100D400068000092690000926E0077278827009261
:100D50007E0000B7086000BF37989FDC8460706138
:100D60007CDCACDDD7DA76DDD5DAD4DA7DDDD4DA39
:100D700086DDD2DAD1DA8DDDD1DA96DDCDDACADAE6
:100D80007F7E70626ADC9ADDA5DCEADCE2DDF5DDFF
:100D900061DDA0DCE5DCDDDDF0DD66DD9BDCE0DCDB
:100DA000D8DDEBDD6CDD96DCDBDCD3DDE6DD71DD93
:100DB00091DCD6DCCEDDE1DD77DD8CDCD1DCC9DD9C
:100DC0000091750010917600083E23E0120710F0A4
:100DD000D4DDD9CF7F7D706440DC02E000936000F9
:100DE000CCDD6CDD77DCBCDCB4DDC7DD33DD72DC93
:100DF000B7DCAFDDC2DD38DD6DDCB2DCAADDBDDD28
:100E00003EDD68DCADDCA5DDB8DD43DD63DCA8DC00
:100E1000A0DDB3DD49DD5EDCA3DC9BDD009160007D
:100E20000A9521F000936000A8DDDBCF7F7B70681E
:100E300014DCA3DD43DD53DC83DC92DCB4DC01E0B5
:100E400000936000C0DC70FF97C0F3DC00DD02DDC2
:100E500046DC76DC85DCA7DCD1DC70FF8DC0E9DC0C
:100E6000F6DC02DD3CDC6CDC7BDC9DDCACDC70FFAA
:100E700083C0DFDCECDC03DD32DC62DC71DC93DCC4
:100E8000BDDC70FF79C0D5DCE2DC03DD28DC58DC9A
:100E900067DC89DC98DC70FF6FC0CBDCD8DC04DD5C
:100EA0001EDC4EDC5DDC7FDCA9DC70FF65C0C1DCD4
:100EB000CEDC04DD14DC44DC53DC75DC0091600026
:100EC0000A9519F000936000BDCFF8948B7F02B3B0
:100ED000077C02BB939AA3E4B1E0FD01789473DC34
:100EE00070FF4AC0A6DC4DDAB2DCF3DCF8DB28DCAC
:100EF00037DC59DC83DC70FF3FC09BDC70DAA7DC99
:100F0000EFDCEDDB1DDC2CDC4EDC5DDC70FF34C087
:100F100090DC86DA9CDCEFDCE2DB12DC21DC43DCFB
:100F20006DDC70FF29C085DCB0DA91DCEBDCD7DB4F
:100F300007DC16DC38DC47DC70FF1EC07ADCE7DA41
:100F400086DCEBDCCCDBFCDB0BDC2DDC57DC57DBA5
:100F500070FF12C06EDC5ADB7ADCE6DCC0DBF0DB53
:100F6000FFDB21DC7F7700917E00013028F40091C7
:100F7000640007FD09F4B3CFE2DC222433244424C7
:040F8000552491CE95
:00000001FF
